:020000040800F2
:10000000C80600208D010008850700088107000848
:1000100083070008810400080511000800000000A3
:10002000000000000000000000000000250B000898
:10003000D50500080000000021080008990B000801
:10004000A7010008A7010008A7010008A7010008F0
:10005000A7010008A7010008D9050008A7010008AA
:10006000A7010008A7010008A7010008A7010008D0
:10007000A7010008A7010008A7010008A7010008C0
:10008000A7010008A7010008A7010008A7010008B0
:10009000A7010008A7010008A7010008A7010008A0
:1000A000A7010008A7010008A7010008A701000890
:1000B000A7010008A7010008A7010008A701000880
:1000C000A7010008A7010008A7010008A701000870
:1000D000A7010008510F0008A7010008A7010008A8
:1000E000A7010008A7010008A701000800F002F816
:1000F00000F03CF80AA090E8000C82448344AAF186
:100100000107DA4501D100F031F8AFF2090EBAE883
:100110000F0013F0010F18BFFB1A43F0010318473B
:10012000F414000014150000103A24BF78C878C1F8
:10013000FAD8520724BF30C830C144BF04680C60ED
:10014000704700000023002400250026103A28BF35
:1001500078C1FBD8520728BF30C148BF0B60704739
:100160001FB501F01AFA1FBD10B510BD00F094F8CC
:100170001146FFF7F5FF01F004FA00F0B2F803B4FE
:10018000FFF7F2FF03BC01F0F9F9000009488047CE
:1001900009480047FEE7FEE7FEE7FEE7FEE7FEE769
:1001A000FEE7FEE7FEE7FEE704480549054A064B81
:1001B00070470000B10B0008ED000008C8000020E7
:1001C000C8060020C8020020C80200207047002096
:1001D00000F03AF8FFF7C8FF012001F0CFF910B5A1
:1001E000203AC0F00B80B1E81850203AA0E818502F
:1001F000B1E81850A0E81850BFF4F5AF5FEA027CF0
:1002000024BFB1E81850A0E8185044BF18C918C05E
:10021000BDE810405FEA827C24BF51F8043B40F8FF
:10022000043B08BF7047D20728BF31F8023B48BFE4
:1002300011F8012B28BF20F8023B48BF00F8012B22
:10024000704770477047704710B500F009F8BDE877
:100250001040AFF30080002801D001F08FB9704743
:1002600010B5002102A000F042F8012010BD0000EE
:10027000534947414252543A2041626E6F726D6158
:100280006C207465726D696E6174696F6E00000038
:1002900000487047640000207546FFF7F9FFAE463E
:1002A00005006946534620F00700854618B020B582
:1002B000FFF77AFFBDE820404FF000064FF000073F
:1002C0004FF000084FF0000B21F00701AC46ACE8FE
:1002D000C009ACE8C009ACE8C009ACE8C0098D466B
:1002E00070470446AFF300802046FFF748FF70B523
:1002F00005460C460A2000E06D1C01F040F935B1BE
:1003000028780028F8D102E0641C01F038F914B113
:1003100020780028F8D1BDE870400A2001F02FB9FC
:1003200000487047680000200029816802D041F031
:10033000010101E021F00101816070470D4910B514
:10034000884202D1012144150AE00B49884202D1BA
:100350000121041504E0094988420AD10121CC0396
:10036000204600F099FA2046BDE81040002100F038
:1003700093BA10BD0024014000280140003C014018
:100380000029816802D041F4801101E021F480113C
:1003900081607047014600208968490700D5012027
:1003A0007047014600208968090700D50120704781
:1003B00010B542680E4B1A40D1E9003442EA0422DB
:1003C0001343436082680B4B1A40D1E90343234334
:1003D0008C6842EA440213438360C26A097D22F4B6
:1003E0007002491EC9B242EA0151C16210BD00004B
:1003F000FFFEF0FFFDF7F1FF70B5072609290AD9C6
:10040000C568A1F10A0404EB4404A640B543A34027
:100410001D43C56007E0056901EB4104A640B543F3
:10042000A3401D4305611F23072A09D2446B521EB6
:1004300002EB820293409C4391400C43446370BDA5
:100440000D2A09D2046BD21F02EB820293409C4317
:1004500091400C43046370BDC46A0D3A02EB820202
:1004600093409C4391400C43C46270BD816841F04D
:10047000080181607047816841F004018160704724
:10048000FEE70000044B01228240186809B11043C6
:1004900000E09043186070470074004010B50121DF
:1004A0004C07204600F0E0F92046BDE8104000214E
:1004B00000F0DAB930B5084C236840F6FE7282408D
:1004C0009343D1E900252A43D1E902510D432A4340
:1004D00082401A43226030BD00740040044A002963
:1004E000516801D0014300E0814351607047000032
:1004F000002004E0016821F0010101600021016099
:1005000041608160C1603149304A0839904203D16D
:10051000486840F00F0006E02C4A1432904204D1A3
:10052000486840F0F00048607047284A28329042FE
:1005300003D1486840F47060F5E7244A3C329042A9
:1005400003D1486840F47040EDE7204A50329042B1
:1005500003D1486840F47020E5E71C4A64329042B9
:1005600003D1486840F47000DDE7184A78329042C1
:1005700003D1486840F07060D5E7154A111F9042DA
:1005800003D1086840F00F0006E0114A143290428F
:1005900004D1086840F0F000086070470C4A283227
:1005A000904203D1086840F47060F5E7084A3C3295
:1005B000904203D1086840F47040EDE7044A50329D
:1005C0009042EAD1086840F47020E5E70800024054
:1005D000080402407047000002490120087000F042
:1005E00003B8000040000020014908607047000087
:1005F0001404014030B51A4AC368016853B3136844
:100600008B431360111D0B680468A3430B604168A2
:1006100011440B68046823430B60114B08331968BD
:100620000468A14319601C1D21680568A943216065
:100630008168102905D011440A68006802430A60E5
:1006400030BD1968026811431960216800680143D0
:10065000216030BD4068104402688A43026030BDAA
:100660000004014010B58A0721F003040649120F67
:1006700021440F238C6893409C438C608B6890408E
:1006800003438B6010BD000000000140F0B58C6892
:10069000002204F00F03E40601D54C6823430C88C4
:1006A0004FF00F0C14F0FF0F4FF0010E1AD0056839
:1006B0000E880EFA02F42640A6420FD196000CFADC
:1006C00006F7BD4303FA06F635438E68282E02D09E
:1006D000482E02D002E0446100E00461521C082A66
:1006E000E6D305600A88FF2A1DD94568002202F179
:1006F00008060EFA06F40E882640A6420FD1960090
:100700000CFA06F725EA070703FA06F58E683D435B
:10071000282E00D144618E68482E00D10461521CFD
:10072000082AE4D34560F0BDF0B5144C002801DA86
:10073000E36900E06368420D120185B2C0F301571E
:100740009540C0F30346032F05D0C2020AD5032209
:10075000B240934307E023F07062636823F0706354
:10076000636002E0AB4343F0706201B12A430028AA
:1007700001DAE261F0BD6260F0BD000000000140FE
:10078000FEE7FEE7FEE7000070B50F24017842683F
:1007900001254FF0E026DAB1124A126802F4E06255
:1007A000C2F5E062120AC2F10403D44042789A40D2
:1007B0008378234013431A010B4BCA54007800F08E
:1007C0001F018D40400906EB8000C0F8005170BD4C
:1007D00001F01F008540480906EB8000C0F88051F9
:1007E00070BD00000CED00E000E400E00A4B1A6868
:1007F00022F0030202431A600848026842F0040231
:100800000260012905D020BF016821F004010160C8
:10081000704730BFF8E700000070004010ED00E0C6
:1008200070470000034A516821F440410143516080
:100830007047000000100240044A0029516901D0AD
:10084000014300E081435161704700000010024005
:10085000044A0029D16901D0014300E08143D161FC
:100860007047000000100240044A0029116901D0BD
:10087000014300E081431161704700000010024015
:10088000044A0029916901D0014300E0814391614C
:100890007047000000100240044A0029D16801D0CE
:1008A000014300E08143D160704700000010024026
:1008B00030B5224A5168224B11F00C0103D00429B3
:1008C00001D0082901D0036015E05168546801F493
:1008D00070114FF0020514F4803F05EB914107D0F1
:1008E000D46A04F00F04641CB3FBF4F34B43EAE74F
:1008F000144B594301605168134B01F0F001090991
:100900005C5C0168E1404160546804F4E064240ADE
:100910001C5D21FA04F48460546804F46054E40A11
:100920001B5DD940C1605268074B02F44042920BF4
:100930001B1F9A5CB1FBF2F1016130BD0010024057
:1009400000127A0000093D00460000200346002006
:100950005909094A01290AD002290AD0516A03F02B
:100960001F02012393400B4200D001207047116801
:10097000F5E7116AF3E70000001002400248406802
:1009800000F00C0070470000001002400B490A689C
:1009900022F480320A600A6822F480220A60B0F5EC
:1009A000803F07D0B0F5802F03D1086840F4A02025
:1009B00008607047086840F48030F9E70010024092
:1009C000014908667047000000004242034A51682E
:1009D00021F0030101435160704700000010024004
:1009E00030B500244FF4A0653120FFF7AFFF641C41
:1009F000AC4201D00028F7D03120FFF7A7FF002834
:100A000000D0012030BD00003EB504460B48012156
:100A100050F82400FFF734FF084869460A3830F8D8
:100A20001400ADF80000102002900320019004484B
:100A300050F82400FFF72AFE3EBD0000BC15000858
:100A4000040000200349044A31F8101052F8200035
:100A500041617047B2150008040000200349044AB0
:100A600031F8101052F8200001617047B2150008EB
:100A700004000020044951F82010CA68034B33F8E1
:100A800010004240CA60704704000020B215000800
:100A900030B5044621480D4689B050F824000121A4
:100AA00040F00100FFF7ECFE042008901B4806A967
:100AB0000C3830F81400ADF81800194850F824002C
:100AC000FFF7E4FD012D27D11448103830F8140049
:100AD000C1B212480E3830F81400C0B2FFF7C2FDA0
:100AE0000E480A3830F814000090002001900820C9
:100AF000CDE902056846FFF77DFD0848083830F863
:100B000014008DF810000F208DF811008DF81200E0
:100B100004A80595FFF738FE09B030BDB8150008E8
:100B200000000020704700001A4900200A6842F4C3
:100B300080320A604FF4A0630A6800F1010012F4E9
:100B4000003F01D19842F7D10868800321D5486859
:100B500048604868486048684860486820F47C10ED
:100B60004860486840F498104860086840F0807019
:100B7000086008688001FCD5486820F003004860E0
:100B8000486840F0020048604868C0F381000228CD
:100B9000FAD17047001002400448407800284FF016
:100BA000000001D0FFF75ABFFFF74CBF4000002004
:100BB000104810B5016841F00101016041680E4A1A
:100BC0001140416001680D4A11400160016821F443
:100BD00080210160416821F4FE0141604FF41F0152
:100BE00081600021C162FFF79FFF05494FF000605F
:100BF000086010BD001002400000FFF8FFFFF6FE85
:100C000008ED00E00029018802D041F0800101E0F8
:100C100021F08001018070470029018802D041F055
:100C2000010101E021F0010101807047002930F845
:100C3000441F02D041F4004101E0C1F30E010180E4
:100C4000704700004B4910B5884202D10121C414FD
:100C500086E0B0F1804F09D0474988420DD101218B
:100C60000220FFF701FE0021022064E00121084676
:100C7000FFF7FAFD002101205DE04049884206D1DE
:100C800001210420FFF7F0FD0021042053E03C493E
:100C9000884206D101210820FFF7E6FD0021082047
:100CA00049E03849884206D101211020FFF7DCFDD8
:100CB000002110203FE03449884206D10121202044
:100CC000FFF7D2FD0021202035E03049884202D1D3
:100CD0000121441444E02E49884202D10121CC0470
:100CE0003EE02C49884202D101210C0538E02A4916
:100CF000884202D101214C0532E02849884206D1C0
:100D000001214020FFF7B0FD0021402013E02449DD
:100D1000884206D101218020FFF7A6FD0021802016
:100D200009E0204988420AD1841501212046FFF7B5
:100D30009BFD00212046BDE81040FFF795BD1A49F4
:100D4000884202D101210C040AE01849884202D1EC
:100D500001214C0404E0164988420AD101218C0487
:100D60002046FFF799FD2046BDE810400021FFF71F
:100D700093BD10BD002C014000040040000800405D
:100D8000000C0040001000400014004000340140FE
:100D9000004C014000500140005401400018004048
:100DA000001C004000200040004001400044014081
:100DB0000048014030B5028C22F010020284028CFF
:100DC0008388048B22F0200224F4E6450C88240654
:100DD00045EA14440D892D0542EA15454A88120555
:100DE00045EA1242104DA84202D0104DA84215D13A
:100DF00022F080054A8923F44063120545EA124235
:100E000022F040058A88120545EA12428D89AD0418
:100E100043EA1545CB899B0445EA13438380048349
:100E2000C9880187028430BD002C01400034014094
:100E300030B5028C22F480520284048C8288838B29
:100E400023F4E6450B881B0645EA134324F40055BA
:100E50000C89240745EA14444D882D0744EA1545BA
:100E6000094CA04202D0094CA04205D122F4804492
:100E70008A89920544EA124282808383C988A0F855
:100E80004010058430BD0000002C014000340140BA
:100E9000828B22F4006242EA0121818370470000C4
:100EA00030B502881B4C1C4DA0420DD0A8420BD07F
:100EB000B0F1804F08D0194B984205D0184B98429A
:100EC00002D0184B984203D122F070034A881A438B
:100ED000154B984206D0154B984203D022F440732C
:100EE000CA881A4302808A8882850A880285A042BD
:100EF0000AD0A84208D00E4A904205D00D4A90422E
:100F000002D00D4A904201D1097A018601218182E5
:100F100030BD0000002C01400034014000040040BE
:100F200000080040000C0040001000400014004089
:100F30000040014000440140004801404FF6FF716D
:100F4000818000210180C1804180017270470000D2
:100F50000E4810B50188890616D5018821F02001B8
:100F60000180011D09880A4CCAB26168094B0B4413
:100F7000491C61601A70712A06D10021616032211A
:100F800000F0B5F80120207010BD000000380140CD
:100F90000C0000205800002010B5028A4FF2FF0319
:100FA0001A400B884C8823438C88C9880C43234300
:100FB0001343038210BD0021018041808180C180E4
:100FC00070470029818902D041F4005101E021F4E9
:100FD000005181817047002A828A01D00A4300E0D3
:100FE0008A43828270470246002012880A4200D05B
:100FF0000120704710B5C1F3421301F01F04012115
:10100000A140012B07D0022B07D01430002A026820
:1010100005D00A4304E00C30F8E71030F6E78A43C5
:10102000026010BD30B50D46018A85B004464CF60D
:10103000FF700140E88808432082A0894EF6F31132
:101040000840A9882A8911436A8902431143A18172
:10105000A18A4FF6FF400140A8890843A082684654
:10106000FFF726FC1B48844201D1039800E0029858
:10107000A1890904002900EBC00101EB00102968D7
:1010800002DA4FEA410101E04FEA8101B0FBF1F0E1
:101090006422B0FBF2F14FEA01114FEA11136FF035
:1010A00018056B4300EB8300A3891D044FF0320346
:1010B00006D503EBC000B0FBF2F000F0070005E03E
:1010C00003EB0010B0FBF2F000F00F0008432081AA
:1010D00005B030BD003801404FF4165101600021C9
:1010E0008180C18001810C2242818181704700B5DD
:1010F0000346C8B2988080211846FFF774FF002885
:10110000F9D000BDFEE70446204600F00FF80221AA
:10111000204600F023FAF7E710B5002100F082F82E
:101120000149016010BD0000FC15000810B5064A19
:1011300000210446117002210120FFF757FB2046D1
:10114000BDE8104000F052B84000002030B58BB030
:1011500001210220FFF77CFB4FF40070ADF81C006A
:10116000182009900220089007A91D48FFF78EFA61
:1011700001211C48FFF7D8FA1B4D2846FFF762FDF6
:1011800042F6E060ADF814004FF47A70ADF810004C
:101190000024ADF81640ADF8124004A92846FFF728
:1011A0007FFE6020ADF800000120ADF8020041F2A2
:1011B0007070ADF80600ADF8084069462846FFF7A4
:1011C00037FE08212846FFF763FE01212846FFF776
:1011D00019FD01212846FFF71FFD0BB030BD0000AF
:1011E00000100140000C1A000004004010B5044635
:1011F0004FF48030FFF7CAFBFFF7F2FBC4F80C0195
:1012000001280DD1FFF7DCFB3920FFF79FFB0028F9
:10121000FAD00220FFF7DAFBFFF7B0FB0828FBD17A
:1012200010BD000010B50C46194902C000F02AF9A3
:1012300000222146FC3000F0E5F805222146001D81
:1012400000F066F8A0F5827472B60020FFF7DCFBB0
:101250000020FFF7F7FB0120FFF7D6FB0120FFF787
:10126000F1FB01210020FFF713FC01210846FFF7E5
:1012700035F901210220FFF731F90121C802FFF7FA
:101280002DF92046FFF762FF62B6204610BD000030
:101290000C16000810B504464FF6FF7088B0814266
:1012A00001D3FEF794FFA1806846FFF747FEA088B0
:1012B000ADF804000C20ADF800000020ADF80600E9
:1012C000ADF8020069462068FFF7EAFD6020ADF83E
:1012D0000C000120ADF80E00A088ADF8120002202D
:1012E000ADF8140003A92068FFF764FD0121206810
:1012F000FFF79CFC08B010BD4FF6FF72914201D37E
:10130000FEF765FF4FF47A725143FFF7C3BF000049
:1013100070B505468AB04FF0804028600C46AA8020
:1013200001214015FFF7ACFA0020FFF77BFA3248A5
:10133000002CD0E9031240690691CDE9072051D075
:10134000012C51D0022C01D0042C4FD00421ADF837
:10135000181006A92948FFF799F9ECB3012C04D01D
:10136000022C02D0042C45D00224254E3046FEF734
:10137000E5FF2149182218316846FEF730FF69461B
:101380003046FFF715F80723012221463046FFF7C4
:1013900033F801213046FEF7F3FF01210846FFF73D
:1013A00057FAA9882846FFF7A7FF01213046FEF724
:1013B000BBFF00212868FFF72FFC3046FFF756F8E7
:1013C0003046FEF7EEFF0028FAD13046FFF753F81B
:1013D0003046FEF7DFFF00E00AE00028F8D10AB04F
:1013E000284670BD4021B2E70221B0E78021AEE778
:1013F0000624BAE70724B8E7C4150008000801402E
:101400000024014030B587B00C460160054601213B
:101410004807FFF71DFAFFF741F81349D1E9000229
:101420008968CDE904020691C4B11020ADF810001E
:1014300004A90E48FFF72AF90022009201920292B5
:1014400003926CB100206946FFF734F854B10020D4
:101450000121FFF717F807B0284630BD2020E5E747
:101460001020F0E71020F3E7C41500080008014041
:1014700010B5044601460248FFF739FE204610BD6C
:10148000003801402DE9F04104468CB0083060601E
:1014900001270026A4F8F86084F8FA703946384627
:1014A000FFF7CAF9012144F20400FFF7E9F9182017
:1014B00002904FF49050DFF89880ADF800000225BC
:1014C000694640460195FFF7E1F8482002904FF445
:1014D0004060ADF80000694640460195FFF7D6F838
:1014E00009A8FFF768FD1B4D09A92846FFF754FD21
:1014F00003A8FFF7F1FD4FF4612003904FF4407013
:10150000ADF8180003A92846FFF78CFD25208DF8BB
:101510001C008DF81E6004208DF81D0007A8089798
:10152000FFF732F9012240F225512846FFF762FD0C
:10153000012280212846FFF74EFD0748FEF7DAFF1B
:1015400001212846FFF73DFD0CB02046BDE8F081A3
:1015500000080140003801404400024029B101293F
:1015600006D0022907D0FEF732FE0120FFF76ABA43
:101570000120FFF773BA0120FFF77CBAFEE700F005
:1015800008B8C4B06846FFF7C7FD6846FFF7BBFD63
:10159000FEE70021C0B2FFF76BBF10B5FEF7C0FE3B
:1015A0004FF00001016010BD0000000001000100CB
:1015B000060000020001000004000000100000000E
:1015C00010000000000000000200000010000000F9
:1015D0000000000003000000000000000000000008
:1015E00000000000000000000000060000000000F5
:1015F00001000000000000000000000000000000EA
:1016000000000000000000000000000000000000DA
:101610000000000034160008000000205800000000
:10162000280100088C1600085800002070060000F1
:101630004401000800080140001001400010014072
:10164000000000000000000004380140000000001D
:1016500010000000000000000000000080000000FA
:10166000000000000000000000000000002000005A
:101670000000000000000204060800000000010253
:0C1680000304010203040607080900002F
:04000005080000ED02
:00000001FF
